:08000000000C05006500AC0CCA
:0800080031002900010C280061
:0800100036092A002A02430709
:08001800100A0E0A0000080A9C
:08002000280C2F000B022C003C
:080028000D022E002500630CFF
:0800300030001A0A3609EC0049
:080038004306AE030E02250091
:080040000B02F0021A0A2C0069
:080048003609630C30000D02C3
:080050002E002500EF0043071C
:080058001A0A650036092A00AE
:080060002A0243071A0A340AC0
:080068000000080A06064A0A1E
:0800700031024307430AE807CF
:08007800580AAC0C310029000C
:08008000010C28000008AC0C83
:0800880031002900010C2800E1
:080090000000000831024307E3
:08009800F100E806540A2902F8
:0800A0004306E800E900000836
:0800A800000000000000000848
:0800B000800CA9000307750A8A
:0800B800460C2D00060CA90006
:0800C00003077F0A640C8900AC
:0800C8000306730A09022B0074
:0800D000AB02010C30002C0012
:0800D8002800AC0C29003100E6
:0800E000290C2F000108640C3B
:0800E800670A08067C0A890C76
:0800F0002D006902A9025E0A5D
:0800F800800C29005C0A060CD3
:08010000E901050C890043062A
:08010800860A330C2D00640C83
:040110002B00670A4F
:0203FE00000AF3
:021FFE00FA0FD8
:00000001FF
